:100000000C946A010C94FE060C94D4060C94AA0677
:100010000C9480060C9456060C942C060C949B01B0
:100020000C949B010C949B010C949B010C949B01E0
:100030000C949B010C949B010C949B010C949B01D0
:100040000C949B010C949B010C949B010C949B01C0
:100050000C949B010C949B010C949B010C94E20565
:100060000C949B010C94AC050C9482050C949B01A0
:100070000C949B010C949B010C949B010C949B0190
:100080000C949B010C949B010C949B010C949B0180
:100090000C949B010C949B010C949B010C949B0170
:1000A0000C949B010C949B010C949B010C949B0160
:1000B0000C949B010C949B010C949B010C949B0150
:1000C0000C949B010C949B010C949B010C949B0140
:1000D0000C949B010C949B010C949B010C949B0130
:1000E0000C949B010C9428030C94D0030C940502EF
:1000F0000C94C2030C94AD030C94D6030C946403CB
:100100000C94780A0C94B1030C94F7010C94DA0364
:100110000C949D010C9428070C94C8030C94A9031B
:100120000C949A030C94DE030C94CC030C9495036A
:100130000C94D4010C94E3010C943D020C94B5038F
:100140000C94E4030C94B8030C94BE030C94E803E1
:100150000C94A5022F0A002300230023005C232314
:1001600023235265616C53696D47656172230000FA
:100170000020002300260029002C002F0032000060
:1001800001000003010601090100000A0B02090C2D
:100190000D0E08070304010000000000000000002D
:1001A000000000000000000000000000000000004F
:1001B000000000000012111000000000000000000C
:1001C000000000000000000000000000000000002F
:1001D000002200250028002B002E003100340002F0
:1001E000010000050108010B010000210024002787
:1001F000002A002D00300033000101000004010737
:10020000010A01050505050705080808080202029C
:10021000020A0A08080404040401010101010101A1
:10022000010303030303030303040707070C0C0C78
:100230000C0C0C0C0C020202020606060606060650
:10024000060B0B0B0B0B0B0B0B01021020200808ED
:100250001020401020408002010201080402010128
:100260000204081020408080402010080402018011
:100270000402018040201008040201080402010168
:100280000204081020408001020408102040802F42
:100290000A002300230023005C23232323526561EB
:1002A0006C53696D4765617223000A003D300A0096
:1002B0003D310A002F0A002300230023005C232382
:1002C00023235265616C53696D4765617223000099
:1002D0002807780A11241FBECFEFD1E2DEBFCDBFC1
:1002E00000E00CBF24E0AAE0B3E001C01D92A33AF5
:1002F000B207E1F713E0A0E0B2E0E2E1FAE100E0EA
:100300000BBF02C007900D92AA30B107D9F711E0D8
:10031000C9E6D1E000E006C021970109802FFE0167
:100320000E94CC0AC836D10780E00807A9F70E94CE
:10033000C0070C94F70C0C940000AF92BF92CF92C0
:10034000DF92EF92FF920F931F93CF93DF936C0195
:100350007B018B01040F151FEB015E01AE18BF0876
:10036000C017D10759F06991D601ED91FC91019028
:10037000F081E02DC6011995892B79F7C501DF9130
:10038000CF911F910F91FF90EF90DF90CF90BF9092
:10039000AF900895E1ECF3E0448155816081718173
:1003A00085E193E00C949D01FC01538D448D252F34
:1003B00030E0842F90E0821B930B541710F0CF96FF
:1003C000089501970895FC01918D828D981761F031
:1003D000A28DAE0FBF2FB11D5D968C91928D9F5F48
:1003E0009F73928F90E008958FEF9FEF0895FC0127
:1003F000918D828D981731F0828DE80FF11D858DDA
:1004000090E008958FEF9FEF0895FC01918D228D6C
:10041000892F90E0805C9F4F821B91098F739927F1
:10042000089585E193E00E94050221E0892B09F4FB
:1004300020E0822F0895FC01A48DA80FB92FB11DD3
:10044000A35ABF4F2C91848D90E001968F7399270A
:10045000848FA689B7892C93A089B1898C918370E8
:1004600080648C93938D848D981306C00288F389E1
:10047000E02D80818F7D80830895EF92FF920F930E
:100480001F93CF93DF93EC0181E0888F9B8D8C8D40
:1004900098131AC0E889F989808185FF15C09FB734
:1004A000F894EE89FF896083E889F98980818370F7
:1004B000806480839FBF81E090E0DF91CF911F91A6
:1004C0000F91FF90EF900895F62E0B8D10E00F5FC7
:1004D0001F4F0F731127E02E8C8D8E110CC00FB69D
:1004E00007FCFACFE889F989808185FFF5CFCE0135
:1004F0000E941B02F1CFEB8DEC0FFD2FF11DE35A93
:10050000FF4FF0829FB7F8940B8FEA89FB898081B7
:100510008062CFCF0F931F93CF93DF938C01D0E0F6
:10052000C0E0F801EC0FFD1F6491662341F085E106
:1005300093E00E943D02892B11F02196F2CFCE016B
:10054000DF91CF911F910F910895CF93DF93EC012D
:10055000888D8823B9F0AA89BB89E889F9898C91AB
:1005600085FD03C0808186FD0DC00FB607FCF7CF67
:100570008C9185FFF2CF808185FFEDCFCE010E9467
:100580001B02E9CFDF91CF9108953FB7F894809196
:10059000110390911203A0911303B091140326B597
:1005A000A89B05C02F3F19F00196A11DB11D3FBFAB
:1005B000BA2FA92F982F8827BC01CD01620F711D7A
:1005C000811D911D42E0660F771F881F991F4A9574
:1005D000D1F708958F929F92AF92BF92CF92DF9200
:1005E000EF92FF924B015C010E94C5026B017C01FE
:1005F0000E94C5026C197D098E099F09683E7340EF
:1006000081059105A8F321E0821A9108A108B1089B
:1006100088EEC80E83E0D81EE11CF11C8114910401
:10062000A104B10429F7FF90EF90DF90CF90BF9025
:10063000AF909F908F9008952FB7F89460910D031D
:1006400070910E0380910F03909110032FBF0895B6
:10065000CF93DF937727FB01E75BFD4F24916D5F1D
:100660007D4FFB0184918823C9F090E0880F991F8A
:10067000FC01E751FE4FA591B491FC01E153FE4FFF
:10068000C591D49141110DC09FB7F8948C912095DC
:1006900082238C938881282328839FBFDF91CF9169
:1006A0000895423051F49FB7F8943C91822F809581
:1006B00083238C93E8812E2BEFCF8FB7F894EC91A6
:1006C0002E2B2C938FBFEACFFC01218930E0F9015A
:1006D000E757FE4F8491F901E75BFD4F94912D5F41
:1006E0003D4FF9012491222309F430C0882311F1F0
:1006F00081508231F8F4E82FF0E08827ED57FC4F65
:100700008F4F0C94CC0AB103B5039503A903AD0335
:100710009A03B803BE03C203C803CC03D003D603B5
:10072000DA039A03DE03E403E803809180008F7705
:1007300080938000E22FF0E0EE0FFF1FE159FE4FA3
:10074000A591B491EC919E2381E009F480E0817041
:100750000895809180008F7DEBCF80918000877F0E
:10076000E7CF84B58F7784BDE5CF84B58F7DFBCF90
:100770008091B0008F778093B000DCCF8091B00083
:100780008F7DF9CF809190008F7780939000D2CFAA
:10079000809190008F7DF9CF80919000877FF5CF79
:1007A0008091A0008F778093A000C4CF8091A0009B
:1007B0008F7DF9CF8091A000877FF5CF80912001B8
:1007C0008F7780932001B6CF809120018F7DF9CF64
:1007D00080912001877FF5CFDC01ED91FD91808133
:1007E000ED91FD919081ED91FD916C9163708E235F
:1007F00009F064609F2309F06860E9E0F4E0E60F27
:10080000F11D659565956D936D917D918D919D918E
:10081000099423C01AC012C016C010C01EC009C05F
:1008200014C013C006C019C009C00DC007C00DC058
:1008300014C062507040804090400BC061507040C6
:100840008040904006C06E5F01C06F5F7F4F8F4F4A
:100850009F4F9E938E937E936E9308958F929F9257
:10086000AF92BF920F931F93CF93DF93CDB7DEB7B5
:10087000A1970FB6F894DEBF0FBECDBF19A24230CC
:1008800008F44AE08E010F5D1F4F842E912CB12C8D
:10089000A12CA50194010E94AA0AE62FB901CA0160
:1008A000EA3044F5E05DD801EE938D01232B242B33
:1008B000252B79F790E080E0109769F0FD01019019
:1008C0000020E9F73197AF014A1B5B0BBD0185E1C1
:1008D00093E00E949D01A1960FB6F894DEBF0FBE73
:1008E000CDBFDF91CF911F910F91BF90AF909F909F
:1008F0008F900895E95CD7CF4AE062E070E080E035
:1009000090E00C942E04009769F0FC010190002007
:10091000E9F73197AF01481B590BBC0185E193E022
:100920000C949D0190E080E0089585E193E00E94A1
:100930000502892BE9F185E193E00E94E3018C3700
:1009400009F58DE591E00E948A028EE592E00E9411
:1009500083048BE591E00E948A020E947C0489E571
:1009600091E00E948A0284E092E00E94830487E57D
:1009700091E00E948A020E94CA0184E591E00E94EF
:100980008A02D3CF8C3329F410920B0310920A03FE
:10099000CCCF8A30C9F380910A0390910B0384363F
:1009A000910594F7019690930B0380930A03BDCFB2
:1009B00008950E94110281110E94950480E090E048
:1009C000892B49F080E090E0892B29F00E940000FB
:1009D00081110E94000080E090E0892B49F080E0C6
:1009E00090E0892B29F00E94000081110E940000F4
:1009F00080E090E0892B49F080E090E0892B29F09D
:100A00000E94000081110C94000008950E94DA0CED
:100A10000F931F93CF93DF93EC0188819981009707
:100A200059F02A813B812617370730F081E0DF91AA
:100A3000CF911F910F9108958B016F5F7F4F0E949F
:100A4000F90B009759F0998388831B830A832C81C3
:100A50003D81232B59F7FC011082E8CF80E0E7CFDE
:100A6000CF93DF93EC0188819981009711F00E9468
:100A7000700B198218821D821C821B821A82DF91E0
:100A8000CF910895EF92FF920F931F93CF93DF932F
:100A9000EC017B018A01BA010E94080581110BC09B
:100AA000CE010E943005CE01DF91CF911F910F91B1
:100AB000FF90EF9008951D830C83B7018881998181
:100AC0000E94F00CF0CFCF93DF93EC01FB0186176F
:100AD000970749F0608171816115710541F044818A
:100AE00055810E944205CE01DF91CF9108950E9469
:100AF0003005F9CFFC0180819181009711F00C94B1
:100B0000700B08951F920F920FB60F9211240BB61F
:100B10000F922F933F934F935F936F937F938F9396
:100B20009F93AF93BF93EF93FF9385E193E00E9470
:100B30001B02FF91EF91BF91AF919F918F917F9198
:100B40006F915F914F913F912F910F900BBE0F903E
:100B50000FBE0F901F9018951F920F920FB60F9215
:100B600011240BB60F922F938F939F93EF93FF93C4
:100B7000E0912503F09126038081E0912B03F09111
:100B80002C0382FD1DC0908180912E038F5F8F7397
:100B900020912F03821741F0E0912E03F0E0EB5EED
:100BA000FC4F958F80932E03FF91EF919F918F9132
:100BB0002F910F900BBE0F900FBE0F901F901895A6
:100BC0008081F2CF1F920F920FB60F9211242F93B4
:100BD0003F938F939F93AF93BF9380910D03909119
:100BE0000E03A0910F03B091100330910C0323E08A
:100BF000230F2D3758F50196A11DB11D20930C032D
:100C000080930D0390930E03A0930F03B0931003F2
:100C10008091110390911203A0911303B0911403DA
:100C20000196A11DB11D8093110390931203A0930F
:100C30001303B0931403BF91AF919F918F913F9194
:100C40002F910F900FBE0F901F90189526E8230F3D
:100C50000296A11DB11DD2CF1F920F920FB60F9217
:100C600011240BB60F922F933F934F935F936F9383
:100C70007F938F939F93AF93BF93EF93FF9390E0F6
:100C800080E00E94EC03FF91EF91BF91AF919F91A3
:100C90008F917F916F915F914F913F912F910F9025
:100CA0000BBE0F900FBE0F901F9018951F920F92C2
:100CB0000FB60F9211240BB60F922F933F934F93C1
:100CC0005F936F937F938F939F93AF93BF93EF93B4
:100CD000FF9390E080E00E94EC03FF91EF91BF91C1
:100CE000AF919F918F917F916F915F914F913F91C4
:100CF0002F910F900BBE0F900FBE0F901F90189565
:100D00001F920F920FB60F9211240BB60F922F93D2
:100D10003F934F935F936F937F938F939F93AF9383
:100D2000BF93EF93FF9390E080E00E94EC03FF916C
:100D3000EF91BF91AF919F918F917F916F915F9153
:100D40004F913F912F910F900BBE0F900FBE0F90C0
:100D50001F9018951F920F920FB60F9211240BB689
:100D60000F922F933F934F935F936F937F938F9344
:100D70009F93AF93BF93EF93FF9390E080E00E9427
:100D8000EC03FF91EF91BF91AF919F918F917F9174
:100D90006F915F914F913F912F910F900BBE0F90EC
:100DA0000FBE0F901F9018951F920F920FB60F92C3
:100DB00011240BB60F922F933F934F935F936F9332
:100DC0007F938F939F93AF93BF93EF93FF9390E0A5
:100DD00080E00E94EC03FF91EF91BF91AF919F9152
:100DE0008F917F916F915F914F913F912F910F90D4
:100DF0000BBE0F900FBE0F901F9018951F920F9271
:100E00000FB60F9211240BB60F922F933F934F936F
:100E10005F936F937F938F939F93AF93BF93EF9362
:100E2000FF9390E080E00E94EC03FF91EF91BF916F
:100E3000AF919F918F917F916F915F914F913F9172
:100E40002F910F900BBE0F900FBE0F901F90189513
:100E5000109218031092170388EE93E0A0E0B0E020
:100E60008093190390931A03A0931B03B0931C0360
:100E700088E492E0909316038093150385EC90E04C
:100E8000909322038093210384EC90E090932403B9
:100E90008093230380EC90E09093260380932503B6
:100EA00081EC90E0909328038093270382EC90E0FC
:100EB00090932A038093290386EC90E090932C036F
:100EC00080932B0310922E0310922F031092300365
:100ED00010923103A2EBB3E090E080E041E2FC012C
:100EE0003E9621E030E08630910510F430E020E0BD
:100EF000E20FF31F40935700E491ED930196893080
:100F0000910569F7E7ECF3E08FE994E04AE050E0FF
:100F10002AE532E0128213821482158257834683B7
:100F2000108631832083118A72968E179F0791F75E
:100F30001092C2031092C1031092C4031092C30313
:100F40001092C6031092C50350E040E061EF72E0DA
:100F500081EC93E00E9442051092BC031092BB0307
:100F60001092BE031092BD031092C0031092BF03F3
:100F70004DE050E065E772E08BEB93E00C944205A6
:100F8000CF93DF93CDB7DEB760970FB6F894DEBF8F
:100F90000FBECDBF789484B5826084BD84B5816076
:100FA00084BD85B5826085BD85B5816085BD809134
:100FB0006E00816080936E001092810080918100AC
:100FC00082608093810080918100816080938100A4
:100FD000809180008160809380008091B100846066
:100FE0008093B1008091B00081608093B0008091C7
:100FF0009100826080939100809191008160809344
:101000009100809190008160809390008091A10078
:1010100082608093A1008091A10081608093A100F3
:101020008091A00081608093A00080912101826066
:101030008093210180912101816080932101809121
:10104000200181608093200180917A0084608093E8
:101050007A0080917A00826080937A0080917A0091
:10106000816080937A0080917A00806880937A0012
:101070001092C100E0912503F091260382E0808365
:10108000E0912103F09122031082E0912303F0917B
:10109000240380E1808310922D03E0912903F091D5
:1010A0002A0386E08083E0912703F0912803808162
:1010B00080618083E0912703F0912803808188601C
:1010C0008083E0912703F0912803808180688083EA
:1010D000E0912703F091280380818F7D808382E354
:1010E00090E0A0E0B0E08093190390931A03A093DE
:1010F0001B03B0931C0368EE73E080E090E00E9455
:10110000EA0243EBC42E43E0D42E8E010F5F1F4F43
:10111000D6018D916D011B861A861D861C861F8641
:101120001E8640E1B80190E00E94800AF80101901B
:101130000020E9F73197AF01401B510BB801CE01F8
:101140000A960E9442051A8219821C821B821E8204
:101150001D8261EC73E0C8010E9463058E859F8546
:10116000AA84BB84ED80FE80E80EF91EA114B104B0
:10117000C9F1892B89F0B701C8010E9408058823AD
:1011800089F129813A818D819E81B501820F931F5A
:101190000E94F00CFE82ED82B80181EC93E00E9487
:1011A0006305C8010E947A05CE010A960E947A055D
:1011B000BBEBCB16B3E0DB0609F0AACF0091C1036D
:1011C0001091C2030115110589F0F801808188236F
:1011D00069F0082E000C990B0E94DF0CD8018D934A
:1011E0008D01F3CFC8010E943005D6CF88E992E087
:1011F0000E948A028EE592E00E94830486E992E0D2
:101200000E948A020E947C0484E992E00E948A0281
:1012100084E092E00E94830482E992E00E948A02C4
:101220000E94CA018FE892E00E948A0227ECE22E17
:1012300023E0F22E04E112E03AE0A32EB12CF801F3
:10124000D0807181D701ED91FC910280F381E02D76
:1012500042E050E06D2DC7011995F701D18A108643
:101260000190F081E02D0190F081E02DC7011995EA
:10127000882339F0D70118968C91189783601896B7
:101280008C930E941C03F70162837383848395838C
:10129000B782A6820C5F1F4FF2E1EF0EF11C8FE9BF
:1012A000E81684E0F80659F67724739492E0692EE4
:1012B0000E941C034B015C0180910A0290910B0279
:1012C000A0910C02B0910D02AC01BD014854544FE5
:1012D0006F4F7F4F84169506A606B70628F488162A
:1012E0009906AA06BB0680F58DEB92E00E948A0261
:1012F0008EE592E00E9483048BEB92E00E948A02CA
:101300000E947C0489EB92E00E948A0284E092E0D1
:101310000E94830487EB92E00E948A020E94CA0125
:1013200084EB92E00E948A0280920A0290920B0261
:10133000A0920C02B0920D028092000290920102E3
:10134000A0920202B092030284E1C82E82E0D82E5D
:1013500007EC13E0D80118968C9118978B7F18969C
:101360008C931897ED91FC910190F081E02DC801CC
:101370001995888BF80180858695817028882816B4
:1013800009F46AC00E941C03D80112966D937D93E4
:101390008D939C93159718968C911897862518967F
:1013A0008C93D80118968C9182FF20C0F60182811F
:1013B00093810E948304D80118969C91892F847090
:1013C00090FD90C0882321F080EB92E00E948A0279
:1013D00064E670E080E090E00E94EA028092000201
:1013E00090920102A0920202B09203020E5E1F4F81
:1013F000B4E0CB0ED11CE016F10609F0ABCF61E0F2
:1014000070E080E090E00E94EA02809100029091FA
:101410000102A0910202B0910302AC01BD014C593E
:101420005F4F6F4F7F4F84169506A606B70628F4C8
:1014300088169906AA06BB0660F48AEA92E00E9422
:101440008A028092000290920102A0920202B0925F
:1014500003020E94D9042CCF0E941C03F8012281B0
:101460003381448155811B012C01221A330A440A1D
:10147000550AB201A10186819781B0E0A0E048172A
:1014800059076A077B0708F48CCF808581703888FC
:10149000381609F486CF0E941C03D80112966D936A
:1014A0007D938D939C93159718968C91189787250B
:1014B000846018968C930E941C03F8012185328564
:1014C00043855485621B730B840B950B6587768768
:1014D0008787908B0E941C03F8016187728783873E
:1014E00094875FCF882309F473CF8CEA92E06ECFA4
:1014F0008BEB93E00E947A0581EC93E00C947A05E3
:10150000BB27FB015527AA27880F991FAA1FA417DD
:1015100010F0A41B83955051B9F7A05DAA3308F0D1
:10152000A95DA193009779F7B111B1931192CB0105
:101530000C949A0ADC01FC01672F71917723E1F783
:10154000329704C07C916D9370836291AE17BF0790
:10155000C8F30895A1E21A2EAA1BBB1BFD010DC002
:10156000AA1FBB1FEE1FFF1FA217B307E407F50753
:1015700020F0A21BB30BE40BF50B661F771F881F2F
:10158000991F1A9469F760957095809590959B01C5
:10159000AC01BD01CF010895EE0FFF1F881F8BBF67
:1015A0000790F691E02D19940F931F93CF93DF933B
:1015B0008230910510F482E090E0E091A104F09176
:1015C000A20430E020E0B0E0A0E0309799F42115CB
:1015D000310509F44AC0281B390B24303105D8F5F0
:1015E0008A819B816115710589F1FB019383828357
:1015F000FE0111C0408151810281138148175907B2
:10160000E0F04817590799F4109761F012960C937F
:10161000129713961C933296CF01DF91CF911F91B1
:101620000F9108950093A1041093A204F4CF211503
:10163000310551F04217530738F0A901DB019A0137
:10164000BD01DF01F801C1CFEF01F9CF9093A204F2
:101650008093A104CDCFFE01E20FF31F81939193FC
:101660002250310939832883D7CF20919F043091AC
:10167000A004232B41F420911002309111023093E9
:10168000A00420939F0420910E0230910F02211597
:10169000310541F42DB73EB740911202509113022B
:1016A000241B350BE0919F04F091A004E217F3078F
:1016B000A0F42E1B3F0B2817390778F0AC014E5FC2
:1016C0005F4F2417350748F04E0F5F1F5093A0045B
:1016D00040939F04819391939FCFF0E0E0E09CCFF3
:1016E000CF93DF930097E9F0FC01329713821282C7
:1016F000A091A104B091A204ED0130E020E0109788
:10170000A1F420813181820F931F20919F04309199
:10171000A0042817390709F061C0F093A004E093F2
:101720009F04DF91CF910895EA01CE17DF07E8F516
:101730004A815B819E0141155105B1F7E901FB83A7
:10174000EA8349915991C40FD51FEC17FD0761F445
:10175000808191810296840F951FE9019983888386
:10176000828193819B838A83F0E0E0E012968D91E1
:101770009C9113970097B9F52D913C911197CD014C
:101780000296820F931F20919F043091A004281786
:10179000390739F6309751F51092A2041092A1043E
:1017A000B093A004A0939F04BCCFD383C283408195
:1017B0005181840F951FC817D90761F44E5F5F4FA1
:1017C00088819981480F591F518340838A819B8169
:1017D000938382832115310509F0B0CFF093A204E1
:1017E000E093A1049ECFFD01DC01C0CF13821282E1
:1017F000D7CF4F925F926F927F928F929F92AF92CC
:10180000BF92CF92DF92EF92FF920F931F93CF93ED
:10181000DF938C01009799F4CB01DF91CF911F9159
:101820000F91FF90EF90DF90CF90BF90AF909F907F
:101830008F907F906F905F904F900C94D40AFC0132
:10184000E60FF71F9C0122503109E217F30708F455
:10185000AEC0D901CD91DC911197C617D70720F101
:10186000C530D10578F0CE0104978617970750F060
:10187000C61BD70B2297C193D1936D937C93CF0155
:101880000E94700BC801DF91CF911F910F91FF90C3
:10189000EF90DF90CF90BF90AF909F908F907F9010
:1018A0006F905F904F9008955B01AC1ABD0A4C0198
:1018B0008C0E9D1EA091A104B091A204512C412C2C
:1018C000F12CE12C109731F580919F049091A004A8
:1018D0008815990509F05CC04616570608F058C0EF
:1018E00080910E0290910F02009741F48DB79EB740
:1018F0004091120250911302841B950BE817F907CF
:1019000008F055C0F093A004E0939F04F90171839F
:101910006083B8CF8D919C91119712966C9012971D
:1019200013967C901397A815B90559F56C0142E000
:10193000C40ED11CCA14DB0420F1AC014A195B09A6
:10194000DA011296159780F0628273825183408388
:10195000D9016D937C93E114F10471F0D7011396D2
:10196000FC93EE9312978ECF22968C0F9D1FF90158
:1019700091838083F301EFCFF093A204E093A1045D
:1019800081CF4816590608F42C017D01D3019ACF66
:10199000CB010E94D40A7C01009749F0AE01B80146
:1019A0000E94E70CC8010E94700B87016BCF10E00A
:1019B00000E068CF81E090E0F8940C94F70C91116E
:1019C000089581568A5108F4805285580895FB0184
:1019D000DC0102C001900D9241505040D8F70895AB
:1019E000FB01DC0101900D920020E1F7089511E068
:1019F000C9E6D1E000E006C0802FFE010E94CC0ABB
:101A00002196011DCA36D10780E00807A9F7F8948E
:021A1000FFCF06
:101A1200FFFFFFFF332E322E3400FFFFFFFF0000D7
:101A2200A30480003100830233008E022D0099024C
:101A32002B00A4022900AF022A00BA022C00C50220
:101A42003000D0023200DB023400E6022800F2024B
:101A52002E00FE02000000003D029D01D401A502FD
:101A62000502E301F7010000000064032803526548
:101A7200616C53696D476561722D47313030304D6D
:101A820046443135003735364536423737363939EF
:101A920039390042544E5F534F46545F310042542D
:101AA2004E5F534F46545F320042544E5F534F468F
:101AB200545F330042544E5F534F46545F340042EA
:101AC200544E5F534F46545F350042544E5F534F5E
:101AD20046545F360042544E5F534F46545F3700C0
:101AE20042544E5F534F46545F380042544E5F5348
:101AF2004F46545F390042544E5F534F46545F3154
:101B0200300042544E5F534F46545F3131004254CD
:0A1B12004E5F534F46545F3132001E
:00000001FF
